:100000000C947D050C949A050C949A050C949A0511
:100010000C949A050C949A050C949A050C949A05E4
:100020000C949A050C949A050C9450290C94222A4D
:100030000C9478230C949A050C949A050C949A05C8
:100040000C949A050C949A050C949A050C949A05B4
:100050000C949A050C9400240C949A050C949A051F
:100060000C949A050C94BD1D0C949A050C949A0559
:100070000C949A050C949A050C949A050C949A0584
:100080000C949A050C949A050C949A050C949A0574
:100090000C949A050C949A050C949A050C949A0564
:1000A0000C949A050C949A050C949A0568096809B1
:1000B00094099409FC091A0A400B400B330ACC0A34
:1000C000DD0ADD0A8F2AB62AAE2BB62AAE2B022B0A
:1000D000252BAE2B7C2B8B2BF100F300F20044453B
:1000E0004255473A2064697361626C65642E0A0068
:1000F00044454255473A20656E61626C65642E0A3C
:10010000000A0025303258006C65645F7461736BBF
:100110003A20004F6E6573686F743A2061637469AA
:1001200076653A2025640A000A0025303862003AD4
:10013000200025303258000A722F632030313233CC
:10014000343536370A00290A002575002F00257539
:10015000005D28002564002000256400200025643F
:100160000020002564007C0025303258006D6F753A
:1001700073656B6579205B62746E7C78207920767C
:1001800020685D287265702F61636C293A205B00DE
:1001900020636F6D6D616E643A2025582C20726566
:1001A00073756C743A2025582C206572726F723A00
:1001B000202558200A00707332206D6F75736520FA
:1001C000656E61626C652064617461207265706F38
:1001D0007274696E67007073325F6D6F7573653A24
:1001E000206661696C20746F20676574206D6F757F
:1001F0007365207061636B65740A002072657375A6
:100200006C743A2025582C206572726F723A202542
:1002100058200A007073325F6D6F7573655F696E89
:1002200069743A207265616420446576494400200F
:10023000726573756C743A2025582C206572726F44
:10024000723A202558200A007073325F6D6F757303
:10025000655F696E69743A20726561642042415439
:100260000020636F6D6D616E643A2025582C2072FA
:100270006573756C743A2025582C206572726F7204
:100280003A202558200A007073325F6D6F757365D0
:100290005F696E69743A2073656E64696E67207277
:1002A0006573657400706275663A2066756C6C0AD9
:1002B00000505332205553415254206572726F7270
:1002C0003A202530325820646174613A202530325A
:1002D000580A00313A0964656C6179282A31306D19
:1002E00073293A2025750A323A09696E7465727667
:1002F000616C286D73293A2025750A333A096D61BE
:10030000785F73706565643A2025750A343A09741C
:10031000696D655F746F5F6D61783A2025750A3588
:100320003A09776865656C5F6D61785F73706565C4
:10033000643A2025750A363A09776865656C5F74FA
:10034000696D655F746F5F6D61783A2025750A008D
:10035000703A097072696E742076616C7565730A03
:10036000643A097365742064656661756C74730A18
:1003700075703A092B310A646E3A092D310A6C7492
:100380003A092B31300A72743A092D31300A45533B
:10039000432F713A09717569740A0A73706565644F
:1003A000203D2064656C7461202A206D61785F7344
:1003B00070656564202A2028726570656174202F3D
:1003C0002074696D655F746F5F6D6178290A776865
:1003D0006572652064656C74613A20637572736F31
:1003E000723D25642C20776865656C3D25640A5351
:1003F000656520687474703A2F2F656E2E77696B6F
:100400006970656469612E6F72672F77696B692FF8
:100410004D6F7573655F6B6579730A004D3E200003
:100420004D25753A25733E20003F0A003D20257575
:100430000A003F0A0064656661756C74730A0025E2
:10044000750A003F0A000A092D2056616C75657314
:10045000202D0A00710A000A092D204D6F75736561
:100460006B6579202D0A003F00433E20004C256437
:100470000A000A092D20537461747573202D0A68CF
:100480006F73745F6B6579626F6172645F6C6564D2
:100490007328293A20253032580A6B6579626F61DA
:1004A00072645F70726F746F636F6C3A20253032C4
:1004B000580A6B6579626F6172645F69646C653A52
:1004C00020253032580A74696D65725F7265616407
:1004D000333228293A202530386C580A000A092D71
:1004E0002056657273696F6E202D0A5649443A2072
:1004F00030783132333428514D4B29205049443A19
:100500002030783536373828545241434B504F49C4
:100510004E542D44454D4F29205645523A203078AF
:10052000303030310A4255494C443A202028466543
:10053000622032372032303232290A4F5054494F2C
:100540004E533A204C554641204D4F5553454B454F
:10055000592045585452414B455920434F4E534F13
:100560004C4520434F4D4D414E44203531320A47D2
:1005700043433A20352E342E30204156522D4C49DB
:1005800042433A20322E302E30204156525F4152A3
:1005900043483A20617672350A000A092D20436FDC
:1005A0006E736F6C65202D0A4553432F713A0971A4
:1005B0007569740A6D3A096D6F7573656B65790AB3
:1005C000000A092D204D61676963202D0A443A090C
:1005D0004465627567204D65737361676520546F6C
:1005E00067676C650A583A094D61747269782044EE
:1005F00065627567204D6F646520546F67676C6531
:10060000202D2053686F77206B6579707265737346
:10061000657320696E206D617472697820677269F4
:10062000640A4B3A094B6579626F617264204465D4
:1006300062756720546F67676C65202D2053686F63
:1006400077206B65797072657373207265706F7255
:10065000740A4D3A094465627567204D6F7573657C
:1006600020546F67676C650A563A0956657273695C
:100670006F6E0A533A095374617475730A433A09E9
:10068000416374697661746520436F6E736F6C6546
:10069000204D6F64650A46312D4631303A09537753
:1006A0006974636820746F204C6179657220302D05
:1006B000392028463130203D204C30290A302D3950
:1006C0003A0953776974636820746F204C617965C7
:1006D0007220302D390A47524156453A09537769FD
:1006E00074636820746F204C617965722030202813
:1006F000616C7465726E617465290A423A094A75C3
:100700006D7020746F20426F6F746C6F61646572DE
:100710000A4553433A094A756D7020746F20426F41
:100720006F746C6F616465722028616C7465726EA1
:10073000617465290A453A095072696E742045450D
:1007400050524F4D2053657474696E67730A42535B
:10075000504143453A09436C65617220454550520A
:100760004F4D0A006B65796D61705F636F6E6669EE
:10077000672E7261773A20253032580A2E737761DE
:10078000705F636F6E74726F6C5F636170736C6FB8
:10079000636B3A2025750A2E636170736C6F636B0F
:1007A0005F746F5F636F6E74726F6C3A2025750AA9
:1007B0002E737761705F6C63746C5F6C6775693AF8
:1007C0002025750A2E737761705F7263746C5F7297
:1007D0006775693A2025750A2E737761705F6C61C1
:1007E0006C745F6C6775693A2025750A2E737761A2
:1007F000705F72616C745F726775693A2025750A63
:100800002E6E6F5F6775693A2025750A2E737761C2
:10081000705F67726176655F6573633A2025750A5C
:100820002E737761705F6261636B736C6173685F75
:100830006261636B73706163653A2025750A2E6E81
:100840006B726F3A2025750A0064656275675F6395
:100850006F6E6669672E7261773A20253032580ACA
:100860002E656E61626C653A2025750A2E6D617485
:100870007269783A2025750A2E6B6579626F61720C
:10088000643A2025750A2E6D6F7573653A202575BB
:100890000A006565636F6E6669673A0A646566613A
:1008A000756C745F6C617965723A2025750A003F3A
:1008B000000A6D6F7573653A206F66660A000A6DEF
:1008C0006F7573653A206F6E0A000A6B6579626F07
:1008D0006172643A206F66660A000A6B6579626F1E
:1008E0006172643A206F6E0A000A6D6174726978F1
:1008F0003A206F66660A000A6D61747269783A2060
:100900006F6E0A000A64656275673A206F66660A50
:10091000000A64656275673A206F6E0A000A0A4A27
:10092000756D70696E6720746F20626F6F746C6F85
:10093000616465722E2E2E2000433E2000436C65BC
:100940006172696E6720454550524F4D0A000A009A
:100950002530325820006B6579626F6172645F7276
:1009600065706F72743A20005B735D005B575D00C9
:100970005B535D005B525D005B445D005B435D006B
:10098000200354005200410043004B0050004F0030
:1009900049004E0054002D00440045004D004F001A
:1009A0000000080351004D004B000000040309043F
:1009B00009025B00030100A0FA0904000001030121
:1009C00001000921110100012240000705810308EF
:1009D00000010904010001030000000921110100C8
:1009E00001227B00070582032000010904020002A6
:1009F00003000000092111010001222200070583E4
:100A0000032000010705030320000112010002007A
:100A1000000008341278560100010200010631FF7F
:100A20000974A1010975150026FF0095207508813C
:100A3000020976150026FF00952075089102C00571
:100A4000010902A10185020901A100050919012975
:100A50000815002501950875018102050109300975
:100A6000311581257F950275088106093815812584
:100A70007F950175088106050C0A38021581257FCE
:100A8000950175088106C0C005010980A101850393
:100A900019012AB700150126B700950175108100CC
:100AA000C0050C0901A101850419012AA002150144
:100AB00026A002950175108100C005010906A1015B
:100AC000050719E029E71500250195087501810240
:100AD0009501750881010507190029FF150026FFFA
:100AE0000095067508810005081901290595057509
:100AF000019102950175039101C011241FBECFEF32
:100B0000DAE0DEBFCDBF11E0A0E0B1E0E8EDF8E54E
:100B100002C005900D92AA3EB107D9F722E0AAEED5
:100B2000B1E001C01D92A73CB207E1F70E94BF16D9
:100B30000C946A2C0C940000FF93EF93E091EA016F
:100B4000F091EB01309709F00995EF91FF9108952D
:100B5000FC018591803011F0EFDFFBCF0895FF2776
:100B6000E0E230E247FF0CC0419597FF09C0EDE29B
:100B70006095709580959095611D711D811D911DE9
:100B800027FF02C0219530E350E2AA27660F771FA6
:100B9000881F991FAA1FA41710F0A41B63955A95CC
:100BA000A9F7AA3008F0A95FA05DAF93F39561158E
:100BB00071058105910541F7ED3211F4EF93F3953D
:100BC000F21718F43F93F395FBCF8F91B5DFFA95A9
:100BD000E1F70895E991F9918591803021F085320E
:100BE00019F0AADFF9CF089520E0E8945591553225
:100BF000C1F3503311F4689455915A3348F450536B
:100C000090F3220F022E220F220F200D250FF4CF7A
:100C10000EF4219589919991533619F3533729F19F
:100C2000533559F1BC0188279927E8945C3621F4A3
:100C30008991999168945591543639F446EF7EF034
:100C400077FF0DC08FEF9FEF0AC055374AE039F0AC
:100C5000583540E121F0523642E009F00895FF9303
:100C6000EF937DDFEF91FF91B7CFFF93EF93FC01FF
:100C700081918030B9F360DFFBCFFF93EF9368DFA2
:100C8000F1CFDF93CF93CDB7DEB72596A3DFCF911A
:100C9000DF91089581E0089581E008950C944C0659
:100CA00008950C9450061F93CF93DF9300D000D08B
:100CB0001F92CDB7DEB749835A836B833091ED0124
:100CC00089819A81311114C0662359F0222349F099
:100CD0000E947D0D182F682F89819A810E94260D10
:100CE00003C00E94510D182F69817A81812F04C0A1
:100CF0000E947D0D69817A810F900F900F900F9067
:100D00000F90DF91CF911F910C949614FC01262F28
:100D1000408151816281738184810C94530681E00A
:100D20000895CF93DF93EC0160E00E948606BE0138
:100D3000DF91CF910C9451060C94E8150C94E415B6
:100D400008950E94D00B0E94A0062FEF84E39CE040
:100D5000215080409040E1F700C000000C94262410
:100D60000F931F93CF93DF938C0161E00E9486065F
:100D7000EC01B8010E944E06882309F45BC0B8015B
:100D8000CE010E940B22882309F454C0B801CE0181
:100D90000E94D719882309F44DC0B801CE010E94E2
:100DA0006721882309F446C0F80182818823D9F19C
:100DB000CF3D8CE5D80779F140F4C115FCE5DF079C
:100DC00091F0C130DC4591F02EC0CC35EDE5DE0769
:100DD00041F1CD35FDE5DF0709F1CB35DD4519F5ED
:100DE0000E94141220C00E94A10624C080915002CB
:100DF000C82FC095C170C0FB80F980935002CC23EE
:100E000029F080EF90E00E94A80514C08EED90E0DC
:100E10000E94A80510C00E94C2120CC00E940B12B2
:100E200002C00E941712C801DF91CF911F910F914C
:100E30000C944A06C0E08C2FDF91CF911F910F9147
:100E400008950E9460230C944C070E944F070C9455
:100E500066238295982F937344E0949F9001112408
:100E60008C7C86958695282B822F8575880F2A7A0B
:100E70002695822B089508950C943B0781E00895F0
:100E80000C943E070895CF93C82F0E943C078C2FE7
:100E90000E944007CF91089580E00C9443070E9480
:100EA00067220C944307CF930E946722C82F80913A
:100EB000EC01C81741F1C093EC018091500282FF10
:100EC0001EC080FF04C088E091E00E94A8058091C8
:100ED000500280FF0CC01F92CF9383E091E09F935C
:100EE0008F930E9441060F900F900F900F9080916A
:100EF000500280FF04C081E091E00E94A8058C2F81
:100F0000CF910C944307CF910895CF93DF93CDB742
:100F1000DEB72B970FB6F894DEBF0FBECDBF4F8361
:100F2000588769877A878B8761110E9443119E01D8
:100F30002F5F3F4F86E0F90111928A95E9F785E02E
:100F4000FE013796D90101900D928A95E1F78981CA
:100F50009A814C815D81452B31F09F3F31F491E0C6
:100F60008F3F19F403C091E001C090E090FF09C0E9
:100F700049815A816B817C818D819E810E946410A0
:100F800005C0C9010E948F068111F2CF2B960FB6C2
:100F9000F894DEBF0FBECDBFDF91CF910895FC0165
:100FA000808191810E94BF0D089570E02091B00270
:100FB0003091B102882319F0622B732B04C0609525
:100FC0007095622373237093B1026093B002089509
:100FD000CF93882309F4A9C0C82F8238C1F40E9496
:100FE000672281FDA2C069E3809102019091030113
:100FF0000E9438230E9465112FEF81EE94E021506A
:1010000080409040E1F700C0000069E319C08338D8
:1010100001F50E94672280FD88C063E5809102018E
:10102000909103010E9438230E9465112FEF81EEF9
:1010300094E0215080409040E1F700C0000063E55B
:1010400080910201909103010E943A23CF910C9468
:1010500065118438C1F40E94672282FD66C067E48E
:1010600080910201909103010E9438230E94651132
:101070002FEF81EE94E0215080409040E1F700C0D6
:10108000000067E4DDCF8CEF8C0F813AF8F48C2FF1
:101090000E941021811149C06C2F80910201909112
:1010A00003010E940223882349F06C2F80910201E2
:1010B000909103010E943A230E9465116C2F809148
:1010C0000201909103010E943823C0CF80E28C0F6F
:1010D000883048F4C77081E001C0880FCA95EAF7EC
:1010E0000E942611B3CFEBE5EC0FE33040F4F0E0C3
:1010F000E95BFE4F808190E0CF910C94CA22E8E535
:10110000EC0FE73150F4F0E0EE0FFF1FE75EFE4F0B
:1011100080819181CF910C94E022CD3E30F08C2FD4
:101120000E944417CF910C941618CF9108958823EC
:1011300009F464C0823879F40E94672281FF5EC09E
:1011400069E380910201909103010E9438230E947B
:10115000651169E310C08338B1F40E94672280FFF3
:101160004DC063E580910201909103010E943823F4
:101170000E94651163E580910201909103010E9434
:101180003A230C946511843879F40E94672282FF17
:1011900035C067E480910201909103010E943823D9
:1011A0000E94651167E4E7CF9CEF980F913A10F425
:1011B000682FE1CF90E2980F983050F4877091E05B
:1011C00001C0990F8A95EAF7892F0E942C11D9CF77
:1011D0009BE5980F933020F480E090E00C94CA22B5
:1011E00098E5980F973120F480E090E00C94E0228D
:1011F0008D3E20F00E949F170C94161808951F939F
:10120000CF93DF93182FEB010E94E807209741F05E
:101210008FE99FE00197F1F700C000002197F6CF1A
:10122000812FDF91CF911F910C949708893319F08A
:1012300060E070E002C060E570E00C94FF08882375
:1012400021F00E9426110C9465110895882321F045
:101250000E942C110C9465110895CF92DF92EF92A9
:10126000FF920F931F93CF93DF937C01D62FC72F4D
:10127000FC011281058102950F700E941C118823C8
:10128000B9F01123A9F08C2F807F803421F080E207
:101290008D0F883068F08091B30282FD09C082E032
:1012A0000E94C5110E941C1191E0D82ED92601C0C0
:1012B000D12CCC2EC2948FE0C8228C2D90E08C30A3
:1012C000910508F0DDC1FC01EA5AFF4F0C94012C96
:1012D0008C2F807FCF70882311F0C295C07F11239F
:1012E00099F0CC2309F4B8C180E28D0F883010F05A
:1012F000D11104C08C2F0E94261103C08C2F0E9494
:1013000036110E946511A8C18D2F0E949708CC2329
:1013100009F4B6C180E28D0F883038F1DD2329F160
:101320008C2F0E943C1124C08C2F807FCF70803284
:1013300011F0C295C07FDD2319F0D130A1F13DC07D
:101340008091B30282FF17C0112349F0CC2329F00A
:101350008C2F0E9426110E94651180E07EC180E0E2
:101360000E949708CC2309F48BC18C2F0E942C116A
:101370000E94651185C1112371F0002341F00130F5
:1013800031F40E9446118C2B0E944E1179C10E94AB
:1013900046118C2B1DC0002319F0013009F470C1D7
:1013A0000E945B1125C0112321F0063008F068C1AE
:1013B0000EC0053008F064C11BC0112361F000238A
:1013C00031F0F701858180FF47C18F7085838C2FB5
:1013D0000E941F0955C1002359F0D93309F04DC1AE
:1013E000FFEF07EE13E0F15000401040E1F743C17A
:1013F0008C2F0E94260944C18C2F86958695837078
:1014000019F0813061F03CC1112321F08D2F9C2F08
:10141000937002C080E090E00E94CA2239C111237B
:1014200021F08D2F9C2F937002C080E090E00E94ED
:10143000E0222EC18D2F112319F00E94441702C003
:101440000E949F178FE08D0F833050F461E070E0B1
:1014500001C0660F8A95EAF7812F0E94D50718C14F
:101460000E94161815C18C2F837009F047C0111106
:101470000BC12D2F229526952770220F220F6D2F3D
:101480006F70862F90E0A0E0B0E0022E04C0880FBD
:10149000991FAA1FBB1F0A94D2F7D4FF10C04FE0B8
:1014A00050E060E070E004C0440F551F661F771FD6
:1014B0002A95D2F7409550956095709503C040E00D
:1014C00050E0BA01C695C695C3708A019B01082BEE
:1014D000192B2A2B3B2BC901B801C23049F058F413
:1014E000C13019F00E943C0CCFC00E942A0CCCC025
:1014F0000E944E0CC9C00E94280CC6C0112319F0CE
:101500008C2F817001C08695882309F4BDC02D2FD2
:10151000229526952770220F220F6D2F6F70862F30
:1015200090E0A0E0B0E0022E04C0880F991FAA1F2F
:10153000BB1F0A94D2F7D4FF10C04FE050E060E028
:1015400070E004C0440F551F661F771F2A95D2F71D
:10155000409550956095709503C040E050E0BA0109
:10156000C695C695C3708A019B01082B192B2A2B9F
:101570003B2BC901B801C23049F058F4C13019F011
:101580000E94010D81C00E94EF0C7EC00E94130DCD
:101590007BC00E94620C78C0CF70112339F08C2F71
:1015A0000E94880C8D2F0E941F096EC08D2F0E94F3
:1015B00026098C2F0E94A90C67C0D23F21F128F484
:1015C000D03F41F0D13FC1F043C0D33F19F1D43FE8
:1015D00079F03EC0112341F0053008F051C08C2F46
:1015E0008F710E94CE0C4CC0063008F049C0F7CF76
:1015F0008091B30282FF18C0112339F08C2F8F71B4
:101600000E94880C3DC01123C9F38C2F8F710E945A
:10161000A90C36C0112329F08C2F8F710E94730CF6
:101620002FC00E946E0C2CC0112349F0CF718C2F5B
:101630000E94880C63E08C2F0E94AA1121C081E0D7
:101640000E94C5110230E0F082E00E94C51118C06E
:10165000112331F0002391F28D2F0E94E80710C072
:10166000002399F2D93349F41FEF27EE33E01150EC
:1016700020403040E1F700C000008D2F0E94970805
:1016800088EF8C0D843020F40E9467220E9443076B
:10169000DD20C9F00E94181180FD15C0F7011282EB
:1016A0000E9412110E94880CC7010E94840B0E94A4
:1016B0001211DF91CF911F910F91FF90EF90DF906A
:1016C000CF900C94A90CDF91CF911F910F91FF90B7
:1016D000EF90DF90CF9008950F931F93CF93DF93F8
:1016E000EC01688179818A810E94CA0D8C010E9477
:1016F000250D0E94160CB801CE010E942D09DF9124
:10170000CF911F910F910895CF93DF93EC019881B2
:1017100089812B813C81232B31F08F3F31F481E093
:101720009F3F19F403C081E001C080E080FD1DC02F
:10173000CE010E94B006811110C00E941C118823A6
:10174000A1F08A81882389F08091B30282FD0DC0C7
:1017500082E0DF91CF910C94C511CE010E946C0BF9
:10176000CE01DF91CF910C949106DF91CF91089536
:1017700080E090E00E94CA2280E090E00E94E02297
:101780000E9443110E9465110E94C9190C941618F9
:1017900080910201909103010E943C230C94B80BAC
:1017A0000E9433110C94C80B92959F70963079F07B
:1017B00010F4925001C09A50923068F4803F69F062
:1017C00018F4883E40F409C0843F29F406C0883EDE
:1017D00020F0813F11F080E0089581E00895FC0140
:1017E000808191810E94BF0D0E94D40B0895CF93F8
:1017F000DF9300D000D01F92CDB7DEB70F900F90CF
:101800000F900F900F90DF91CF910895CF93DF93BA
:1018100000D000D000D0CDB7DEB726960FB6F89432
:10182000DEBF0FBECDBFDF91CF910895089508951B
:101830000C94170C0C94180C0E941A0C6093F7016E
:101840007093F8018093F9019093FA010C94B80B0E
:101850000C941C0C0F931F930091F7011091F80149
:101860002091F9013091FA01602B712B822B932B7F
:101870001F910F910C941C0C0F931F930091F70173
:101880001091F8012091F9013091FA016023712340
:10189000822393231F910F910C941C0C0F931F9381
:1018A0000091F7011091F8012091F9013091FA01AE
:1018B00060277127822793271F910F910C941C0C8E
:1018C0000C94170C0E94600C6093F3017093F40168
:1018D0008093F5019093F6010C94B80B60E070E0F2
:1018E000CB010C94620C0F931F9341E050E060E039
:1018F00070E08A019B0104C0000F111F221F331FDB
:101900008A95D2F7C901B8011F910F910C94620C0E
:101910000F931F9341E050E060E070E004C0440F7B
:10192000551F661F771F8A95D2F78091F30190911A
:10193000F401A091F501B091F6018A019B01082BF9
:10194000192B2A2B3B2BC901B8011F910F910C9425
:10195000620C0F931F9341E050E060E070E004C020
:10196000440F551F661F771F8A95D2F740955095F3
:10197000609570958091F3019091F401A091F5012B
:10198000B091F6018A019B01082319232A233B23E6
:10199000C901B8011F910F910C94620C0F931F9312
:1019A00041E050E060E070E004C0440F551F661F46
:1019B000771F8A95D2F78091F3019091F401A0915D
:1019C000F501B091F6018A019B01082719272A2702
:1019D0003B27C901B8011F910F910C94620C0F9322
:1019E0001F930091F3011091F4012091F5013091C2
:1019F000F601602B712B822B932B1F910F910C946E
:101A0000620C0F931F930091F3011091F401209148
:101A1000F5013091F60160237123822393231F91F6
:101A20000F910C94620C0F931F930091F30110918E
:101A3000F4012091F5013091F6016027712782278A
:101A400093271F910F910C94620C0895292F220F58
:101A5000920F890FE82FE695E695E695877051E09D
:101A600001C0550F8A95EAF785E0E89FF00111243F
:101A7000E251FE4F20E030E070E04081CB01022EC9
:101A800002C0969587950A94E2F781708195842724
:101A90008523842781932F5F3F4F2530310569F7D8
:101AA0000895292F220F920F890F682F669566954A
:101AB0006695982F977085E0689FB001112440E0EB
:101AC00050E080E0FB01E40FF51FE251FE4F208162
:101AD00030E0092E02C0369527950A94E2F721706E
:101AE0003327042E01C0220F0A94EAF7822B4F5F9E
:101AF0005F4F4530510531F70895BF92CF92DF9285
:101B0000EF92FF920F931F93CF93DF938C01C090BE
:101B1000F301D090F401E090F501F090F60180918E
:101B2000F7019091F801A091F901B091FA01C82A4A
:101B3000D92AEA2AFB2ACFE1D0E0D701C6010C2E30
:101B400004C0B695A795979587950A94D2F780FD1E
:101B500004C0219790F7B12C07C0BC2EB8018C2F80
:101B60000E94AA140197A9F38B2DDF91CF911F91A9
:101B70000F91FF90EF90DF90CF90BF900895CF939B
:101B8000DF93EC010E947D0DBE010E94AA14DF913B
:101B9000CF9108951F93CF93DF93EB019091ED01C7
:101BA000992321F0CB010E94BF0D13C0882349F077
:101BB000CB010E947D0D182F682FCE010E94260DAB
:101BC00004C0CB010E94510D182FBE01812F0E942D
:101BD000AA14DF91CF911F9108951F93CF93DF93A4
:101BE000C091FB0116E08091FC01C81799F0D0E08C
:101BF0001C9FF0011D9FF00D1124E350FE4F40810A
:101C0000518162817381848195810E94060C2196A5
:101C1000C770E9CFDF91CF911F91089540912D02B8
:101C200050912E0260912F0270913002809131020A
:101C3000909132020C94060CEF92FF920F931F9337
:101C4000CF93DF938091320282958F7009F065C047
:101C500080912F02882309F460C08091FB01F090ED
:101C6000FC0110912D0200912E02609130027091C2
:101C7000310291E01F3F09F090E0C0910001D09146
:101C80000101292F96E0E92E8F1509F446C0611550
:101C9000710521F00F3F21F030E003C031E001C0B9
:101CA000322F90E030FD36C0E89EF001E99EF00D45
:101CB0001124DF01A350BE4F11963C9111973013B0
:101CC00029C03C91311326C012963C9112973111D4
:101CD00021C013964D915C911497461B570B4C17DE
:101CE0005D07C0F4809132028F7080618093320270
:101CF000EE5FFD4F80818F70806180838DE292E086
:101D00000E94840BDF91CF911F910F91FF90EF9074
:101D10000C94ED0D01968770B7CFDF91CF911F9195
:101D20000F91FF90EF9008959F92AF92BF92CF9244
:101D3000DF92EF92FF920F931F93CF93DF93CDB774
:101D4000DEB761970FB6F894DEBF0FBECDBF8C0132
:101D500085E0F801DE011D9601900D928A95E1F76C
:101D6000D8011296EC9090912D02E0912E022091D4
:101D70003002309131022115310531F0EF3F31F45D
:101D800081E09F3F19F403C081E001C080E0B82FDB
:101D9000B1709B2E80FD47C1D8014C9111965C918A
:101DA00011971396AD90BC9014978DE2C82E82E0E7
:101DB000D82EF0902F02B501621B730B2091000109
:101DC00030910101FF2009F4D9C0809132026217DD
:101DD000730708F095C0282F207F09F052C05E13CA
:101DE00013C0491311C0FE2CE1100EC08F7080612A
:101DF000809332020E940E0EC6010E94840B8091D5
:101E00003202F80185834DC1AB2831F05F3F31F4D8
:101E100081E04F3F19F403C081E001C080E080FD04
:101E200003C081E08E2502C080E090E0F82FF170C1
:101E3000FF2E80FF1CC08091FB012091FC0136E049
:101E4000821709F40BC190E0389FF001399FF00D23
:101E50001124E350FE4F6181561306C06081461382
:101E600003C06281E61203C001968770E9CFFE2CA1
:101E7000EE2009F416C18091320281608093320213
:101E800054C05E1306C0491304C0E11002C0F8013B
:101E900099C0C8010E94EF0B882361F1EE2051F137
:101EA00020913202822F82958F7090E0029774F019
:101EB00080912D0290912E0298878F831986BB8680
:101EC000AA862C87CE0107960E94840B86E0F80133
:101ED000ADE2B2E001900D928A95E1F70E941C0EEE
:101EE0000E940E0E0AC05E1711F1C8010E94EF0B8E
:101EF00081112CC0C8010E94840BFF24F394D1C02F
:101F0000282F207F81F77A2DB98AA88A6E2D89899A
:101F10000E94F70B8DE292E00E94840B86E0D601CE
:101F20001D928A95E9F70E940E0EF12CBAC0491352
:101F3000DCCFE110DACFF8018583C8010E94840B61
:101F400086E0D6011D928A95E9F7ABC0EE2091F2AA
:101F500020913202822F82958F7090E002970CF4CC
:101F6000B5CF80912D0290912E029A8389831B8296
:101F7000BD82AC822E83CE010196A6CF6217730775
:101F800008F044C0FE2CEE2009F4B4CF5E1330C03C
:101F900049132EC02091320220FD21C0822F82954C
:101FA0008F70482F50E041155105C9F0F801258385
:101FB0004F30510541F08F5F982F9295907F822F7F
:101FC0008F70892B8583C8010E94840B86E0F801FD
:101FD000ADE2B2E001900D928A95E1F73CC086E057
:101FE000F801ADE2B2E001900D928A95E1F759C097
:101FF000C8010E94EF0B811169CF8091320281608C
:1020000080933202C8010E94840B4BC07A2DB98A9A
:10201000A88A6E2D89890E94F70B86E0D6011D9251
:102020008A95E9F718C0EE2009F464CFC8010E9430
:10203000EF0BF82E882309F45DCF86E0F801ADE2BE
:10204000B2E001900D928A95E1F78DE292E00E9454
:10205000CF070E941C0E0E940E0E23C04D875E8784
:102060008D859E850E94BF0D292F22952F702230CD
:1020700028F49F7039F0811105C00BC0243028F47A
:102080009F7049F4805E883020F0C8010E94840B64
:102090009F2CF92C06C0D80115969C91907F91F742
:1020A000F8CF8F2D61960FB6F894DEBF0FBECDBF6F
:1020B000DF91CF911F910F91FF90EF90DF90CF9024
:1020C000BF90AF909F9008951F93CF93DF93CDB7AC
:1020D000DEB72C970FB6F894DEBF0FBECDBF4F838F
:1020E000588769877A878B879C87CE0107960E94DD
:1020F000940E8823D1F09F8188852A853B85232BE8
:1021000031F08F3F31F481E09F3F19F403C081E04B
:1021100001C080E080FD47C04F81588569857A8580
:102120008B859C850E94060C3EC086E0FE0137969A
:10213000DE01119601900D928A95E1F7FF81E88505
:102140006A857B856115710531F0EF3F31F481E0DF
:10215000FF3F19F403C081E001C080E080FD23C08F
:102160002091FC0130E0C9010196877099274091C8
:10217000FB0150E084179507F1F1F983EA837D8331
:102180006C8396E0929FD001939FB00D1124A350D1
:10219000BE4FFE01319601900D929A95E1F7809322
:1021A000FC010E94ED0D16E08091FB019091FC0175
:1021B000891771F1189FC001112483509E4F0E940E
:1021C000940E882329F1E091FB011E9FF001112458
:1021D000E350FE4F408151816281738184819581FA
:1021E0000E94060C8091FB0190E001968770992770
:1021F0008093FB01D9CF0E94D00B1092FC0110926A
:10220000FB01EDE2F2E086E0DF011D928A95E9F73D
:102210002C960FB6F894DEBF0FBECDBFDF91CF91E5
:102220001F91089580913B02859585958595089528
:1022300080913B028770089590913B02977081E0F6
:1022400009F480E008958091460208959091460235
:10225000892B8093460208958095909146028923A8
:102260008093460208951092460208959091450287
:10227000892B80934502089580959091450289238A
:1022800080934502089510924502089580913C0282
:10229000089508950C9449110C944A119091B30239
:1022A00092FD08C090913C02981721F080933C0267
:1022B0000C944C11089580913C02882329F01092CF
:1022C0003C0280E00C944C110895CF93DF93E09191
:1022D0000201F0910301809146028083E0910201A6
:1022E000F0910301908180914502892B8083809138
:1022F0003C02882381F0E0910201F091030190817A
:10230000892B808380910201909103010E94F62223
:1023100081110E945B11C0910201D091030148E03C
:1023200050E063E372E0CE010E941B2C892B69F020
:1023300088E0FE01A3E3B2E001900D928A95E1F7F7
:10234000CE01DF91CF910C947322DF91CF9108954C
:102350000C9449119091B30292FD10C098E0899FAE
:1023600090011124262B20933B020E94880C80911F
:102370003B028595859585950C94A8110C94880C45
:1023800010923B0280E00C94A81120913B028095B2
:10239000822380933B02982F977099F430E0482F66
:1023A000082E000C550B2417350759F09091B302F5
:1023B00092FD07C08595859585950E94A90C0C9482
:1023C000C0110895CF939091B30292FB222720F978
:1023D0002817F9F0C82F892FC0FB82F98093B30228
:1023E0008091B2029091B3020E943E1282E00E945C
:1023F000C5118091500280FF0CC01F92CF9383E1E2
:1024000091E09F938F930E9441060F900F900F9041
:102410000F90CF9108958091B30282FB882780F9B5
:1024200091E089270C94E21181E00C94E21180E0A4
:102430000C94E21180E090E00E94302C21E0893E73
:102440009E4F09F020E0822F089582E090E00C94E6
:10245000282C83E090E00C94282CCF9384E090E02B
:102460000E94282CC82F82E290E00E94282C2C2F5A
:1024700030E0A901582BCA01CF910895CF93C92FFD
:10248000682F84E090E00E94362C6C2F82E290E06E
:10249000CF910C94362CAB01BC018FE090E00C94F2
:1024A000482CAB01BC0183E190E00C94482C60E027
:1024B00070E0CB010C94511260E070E0CB010E94FF
:1024C0004B120C94571269EE7EEF80E090E00E9470
:1024D000542C60E082E090E00E94362C60E083E0C3
:1024E00090E00E94362C1092F7011092F8011092A1
:1024F000F9011092FA0160E084E090E00E94362C2D
:1025000060E082E290E00E94362C60E085E090E09E
:102510000E94362C60E086E090E00E94362C6FEF3F
:1025200087E090E00E94362C40E050E0BA0188E05D
:1025300090E00E94482C60E08DE090E00E94362CF4
:1025400040E050E0BA0188E190E00E94482C60E051
:1025500087E190E00E94362C40E050E0BA018CE127
:1025600090E00E94482C60E070E080E290E00E94E1
:10257000542C40E050E0BA0188E190E00E94482CE1
:102580000C945C120C946312682F8EE090E00C9413
:10259000362C0E94E52360934C0270934D02809389
:1025A0004E0290934F0260934802709349028093C9
:1025B0004A0290934B02089585B7806885BF85B71E
:1025C000806885BF089581E008950C94E312089512
:1025D0000C94E7120C94E7120C94EA120C94E71294
:1025E0000C94EE120C94E7120E94DC128BE296E23D
:1025F0000E945D220E94F2120C94F0120E94E812D6
:102600000C94E7120E9487150C9442070E94D02375
:102610000E944B160E9402130E94161C0C94EC128E
:10262000DF92EF92FF920F931F93CF93DF93CDB77B
:10263000DEB72A970FB6F894DEBF0FBECDBF0E945B
:102640005616D82E81110E94C91280E00E94AB1547
:10265000F82EE0904702E82689F48FEF89838A8379
:102660001B820E94D9238160782F9D838C834981AE
:102670005A816B818D810E9485072CC08091500208
:1026800081FD0E94B11500E011E08E2D8123E9F05B
:102690000E94E512882399F00E831F82F12281E0C7
:1026A00009F480E088870E94D9238160782F9A8777
:1026B00089874E815F8168858A850E948507809120
:1026C000470218271093470205C00F5F110F033010
:1026D000E1F6C3CF81E0D11001C080E02A960FB6A9
:1026E000F894DEBF0FBECDBFDF91CF911F910F9148
:1026F000FF90EF90DF9008950E9410130E94B6188B
:102700000E94211B0C945307CF93DF930E94AF14B8
:10271000EC01811521E5920708F045C0811530E5EF
:10272000930708F094C0883E910528F5803E9105F6
:1027300008F0F8C0883A910570F4853A910508F0E0
:102740007CC08130910509F475C008F4E8C0049795
:1027500008F0E8C0E4C08F3B910508F0E0C0C85A1B
:10276000D0E0CC0FDD1FC65BDE4F0990D881C02DB5
:10277000CE019464D8C0811540E2940758F48115C5
:1027800051E0950708F0CEC08D3E910508F4C7C012
:102790009065C9C0C11580E4D80708F4C0C0DF70D7
:1027A000CE01906AC0C0811525E59207A8F4811575
:1027B00034E5930708F095C0811543E5940708F0C8
:1027C0007BC0811552E5950708F061C0D82FCC2752
:1027D000CE01816F906AA7C0C11589E5D807A0F422
:1027E000C11528E5D20708F082C0C11536E5D30728
:1027F00008F095C08C2F0E9443158F7190E0D82F60
:10280000CC27CE0190628FC0C1154AE5D40708F4E9
:1028100074C0CE0190568115904208F080C08D2F73
:102820008F710E944315DD27D0628F71AE01582B46
:10283000CA0179C081E090E076C0C55AD0E0C8589E
:10284000DE4F8881C82FD0E0CE0190646CC074E068
:10285000969587957A95E1F7282F23703C2F337052
:1028600081E090E002C0880F991F3A95E2F79C68DA
:10287000AC01522B9A019C2F9F709695969550E231
:10288000959FE0011124C9018C2B9D2B4CC08370B6
:10289000992721E030E002C0220F331F8A95E2F72A
:1028A0009C2F9695969580E2989FE0011124C22B6B
:1028B000D32BCE019C6837C08370992721E030E08C
:1028C00002C0220F331F8A95E2F79C2F96959695AA
:1028D00040E2949FE0011124C22BD32BCE019A68D1
:1028E00022C0D82FCC27CE01846F906A1CC0DC2F69
:1028F000CC27CE01806F906A16C08C2F8F700E94FB
:10290000431594E0D695C7959A95E1F7CF70D0E03E
:10291000DC2FCC27D0699E01282BC90104C080E0A0
:1029200090E001C0CE01DF91CF910895E72FF0E054
:102930009F01280F311DC901F901EE0FFF1FE80F9C
:10294000F91FE60FF11DEE0FFF1FE852FF4F8591B3
:10295000949108950E9496140E94841308958238D9
:10296000910569F1B0F48133910509F46DC048F423
:102970008932910509F463C08A32910509F469C06E
:1029800008958533910509F455C089339105B9F04F
:102990000895833E910569F138F4803E9105B1F0C8
:1029A000823E910509F10895863E9105A9F1873E81
:1029B0009105B9F1843E910509F064C023C02091CE
:1029C000B20220FD4FC021FD4DC008958091B2029A
:1029D00080FD44C08091B30280FF44C08091B20268
:1029E00084FD42C083EE4DC08091B20282FF38C0A8
:1029F000F5CF8091B20282FD33C08091B30280FD99
:102A000031C0ECCF8091B30281FF32C08091B2021D
:102A100084FD2AC087EE35C08091B20283FF26C0B4
:102A2000F5CF8091B20283FD21C08091B30281FD78
:102A30001FC0ECCF8091B20285FD1CC01DC08091EB
:102A4000B20285FD19C016C08091B20286FD16C083
:102A500017C08091B20286FD13C010C089E311C077
:102A600082EE0FC080EE0DC080E00BC086EE09C084
:102A700084EE07C089E205C085E303C08AE201C095
:102A800081E390E008959091B20292FF0DC0282F4B
:102A90002871283019F4877F846006C0282F24719C
:102AA000243011F48B7F886093FF0DC0282F28718C
:102AB000283119F4877E846106C0282F24712431BF
:102AC00011F48B7E88612091B30220FF0DC0382F56
:102AD0003871383019F4877F816006C0382F317122
:102AE000313011F48E7F886021FF0DC0282F2871AE
:102AF000283119F4877E816106C0282F2171213188
:102B000011F48E7E886194FD877E089508950E9459
:102B10001A12811102C00E94C2120E9425128093D3
:102B200050020E942D129093B3028093B2020E9431
:102B300086150E942912682F70E080E090E00E94C4
:102B4000280C6091F3017091F4018091F50190914E
:102B5000F6010C94600CE82FF0E0EB54FD4F8081FF
:102B6000089587E391E00E94A8051F921F9282E3D7
:102B700091E09F938F930E9441068FE291E00E9423
:102B8000A8058091B5020E9429071F928F938AE2BF
:102B900091E09F938F930E9441068DB79EB7089650
:102BA0000FB6F8949EBF0FBE8DBF88E291E00C94E3
:102BB000A80580EA8A95F1F7089500C008950C945D
:102BC000D91508950C94E1150C94E2150C94E115B7
:102BD0000C94E615F894E82FE295EF70F0E031A13F
:102BE000282F2F7081E090E001C0880F2A95EAF726
:102BF000982F9095932391A392A1892B82A37894E7
:102C0000089580EF0E94EA1581EF0E94EA1584EF93
:102C10000E94EA1585EF0C94EA150F931F93CF934A
:102C2000DF938C01D62FF894809A889878940E942C
:102C3000DD15EBE7F1E031E0C0E021912F3F89F0B5
:102C4000A22FA295AF70B0E090968C9190E02F707B
:102C500002C0959587952A95E2F780FD02C0832FE3
:102C600001C080E0C82B330F81E0EE37F80729F769
:102C700080EF0E94EA1561E0C11101C060E08D2F74
:102C80000E94DF15F801ED0FF11DC083DF91CF9198
:102C90001F910F9108950E9401161092B502109293
:102CA000B40281E00E947C160C949C061F93CF9383
:102CB000DF931F92CDB7DEB7198260E0CE01019697
:102CC0000E940D169091B402898111E0981301C001
:102CD00010E098138093B402212F41E065EB72E07D
:102CE00084EB92E00E947D160E949E06812F0F9039
:102CF000DF91CF911F9108950895FF920F931F9335
:102D0000CF93DF938C01F62ED72FC42F222349F0C7
:102D100081E0809353020E94D923909352028093C2
:102D20005102809153028823C1F080915102909109
:102D300052020E94F123059780F0EF2DFD2FD8015C
:102D40004C2F50E0CD01801B910B841795071CF48C
:102D50008D918193F7CF10925302DF91CF911F9104
:102D60000F91FF9008950E94A7260E9406130C94CD
:102D7000B3260E94B7260E947C130C94D5260E948D
:102D800077230E948E260E94F4120E94B3160E949E
:102D9000B9160E94FE12FBCF80915A0280FF06C036
:102DA0006091090170E0660F771F26C081FF04C0A3
:102DB0006091090184E005C082FF07C060910901AC
:102DC00088E0689FB001112417C09091590299239F
:102DD000D1F060910801961788F72091090188E0E9
:102DE000289F90011124929FA001939F500D1124C0
:102DF00070E0CA010E94ED2B6038710540F4611546
:102E0000710519F406C068E070E0862F08958FE719
:102E1000089581E0089580915A0280FF08C0609172
:102E2000050170E0759567957595679521C081FFDF
:102E300006C06091050170E07595679519C082FF25
:102E400004C06091050170E010C090915802992370
:102E500099F0609104019617A0F780910501899F70
:102E6000C001112470E00E94ED2B6038710540F420
:102E70006115710519F406C061E070E0862F0895B0
:102E80008FE7089581E008958D3E21F40E94CC16CD
:102E9000819504C08E3E29F40E94CC1680935E0278
:102EA00008958F3E21F40E94CC16819504C0803F86
:102EB00029F40E94CC1680935D020895893F19F48D
:102EC0000E940B1705C08A3F31F40E940B178195B1
:102ED00080935F0208958B3F21F40E940B17819528
:102EE00004C08C3F29F40E940B1780936002089560
:102EF0009FE0980F983078F421E030E0A90102C0FB
:102F0000440F551F9A95E2F7CA0190915C02892BF4
:102F100080935C0208958D3F21F480915A02816074
:102F20000BC08E3F21F480915A02826005C08F3F12
:102F300029F480915A02846080935A0208958D3E4C
:102F400039F490915E0297FF35C010925E0259C02D
:102F50008E3E29F490915E021916BCF32BC090911D
:102F60005D028F3E29F497FF25C010925D0249C093
:102F7000803F19F41916CCF31DC090915F02893F70
:102F800029F41916BCF410925F023BC08A3F19F471
:102F900097FF10C0F8CF8B3F39F49091600297FFF4
:102FA00009C0109260022DC08C3F21F49091600204
:102FB0001916BCF39FE0980F983080F421E030E0C0
:102FC000A90102C0440F551F9A95E2F7CA018095E6
:102FD00090915C02892380935C0213C08D3F21F4A1
:102FE00080915A028E7F0BC08E3F21F480915A024D
:102FF0008D7F05C08F3F29F480915A028B7F80938B
:103000005A0280915D02811106C080915E02811199
:1030100002C01092590280915F02811106C0809116
:103020006002811102C010925802089580915002EE
:1030300083FF7EC08DE691E00E94A80580915C022E
:103040001F928F9388E691E09F938F930E94410691
:1030500086E691E00E94A80580915D02282F082E47
:10306000000C330B3F938F9383E691E09F938F93F4
:103070000E94410681E691E00E94A80580915E02CF
:10308000282F082E000C330B3F938F938EE591E091
:103090009F938F930E9441068CE591E00E94A805C2
:1030A00080915F02282F082E000C330B3F938F93E3
:1030B00089E591E09F938F930E94410687E591E017
:1030C0000E94A80580916002282F082E000C330B67
:1030D0003F938F9384E591E09F938F930E944106E5
:1030E00081E591E00E94A805809159021F928F937B
:1030F0008EE491E09F938F930E9441068CE491E0CF
:103100000E94A80580915A021F928F9389E491E052
:103110009F938F930E94410686E491E00E94A80548
:103120008DB79EB74C960FB6F8949EBF0FBE8DBF5D
:103130000E94D92320915D02211104C020915E02DA
:10314000222321F0909357028093560220915F0230
:10315000211104C020916002222321F09093550296
:10316000809354028BE592E00C94BC22EF92FF9284
:103170000F931F93CF93DF9300D000D000D0CDB733
:10318000DEB786E0EBE5F2E0DE01119601900D92EC
:103190008A95E1F7E0905D02F0905E0200915F0297
:1031A0001091600210925D0210925E0210925F0216
:1031B00010926002E11003C0FF2009F45DC080910D
:1031C0005602909157020E94F123AC01909159024E
:1031D000992339F020910A0130E02417350758F07F
:1031E0004BC020910B018AE0289F900111242417E5
:1031F000350718F041C09F3F19F09F5F9093590227
:10320000EE2061F00E94CC161E1414F09FEF01C056
:1032100091E0989F902D112490935D02FF2061F022
:103220000E94CC161F1414F09FEF01C091E0989FEC
:10323000902D112490935E0230915D023323E1F0D2
:1032400020915E022223C1F045EB3403C00111241A
:10325000992319F090935D0203C081E080935D0291
:1032600035EB2303C0011124992319F090935E02DA
:1032700003C081E080935E02011103C0112309F4B1
:103280005DC080915402909155020E94F123AC01DF
:1032900090915802992339F02091060130E02417CB
:1032A000350758F04BC0209107018AE0289F900114
:1032B00011242417350718F041C09F3F19F09F5F74
:1032C00090935802002361F00E940B17101614F01F
:1032D0009FEF01C091E0989F902D112490935F0281
:1032E000112361F00E940B17111614F09FEF01C01B
:1032F00091E0989F902D11249093600230915F028D
:103300003323E1F0209160022223C1F045EB340326
:10331000C0011124992319F090935F0203C081E04A
:1033200080935F0235EB2303C0011124992319F028
:103330009093600203C081E08093600280915D02FF
:1033400081110BC080915E02811107C080915F02E4
:10335000811103C08091600281110E941618EB82D6
:10336000FC820D831E8386E0FE013196ABE5B2E060
:1033700001900D928A95E1F726960FB6F894DEBF7C
:103380000FBECDBFDF91CF911F910F91FF90EF90B6
:103390000895EBE5F2E086E0DF011D928A95E9F7FA
:1033A000109259021092580210925A020895CF9327
:1033B000DF93EC01FB018281882309F43CC1C43016
:1033C000FDE5DF0760F4CB3F9CE5D90788F49E015B
:1033D00022503C452431310508F02EC109C0C236C7
:1033E000EDE5DE0729F0C63AFDE5DF0709F024C167
:1033F0000E942D129093B3028093B202C1318CE5EA
:10340000D80709F4C6C008F042C0C930ECE5DE07B1
:1034100009F49BC000F5C5308CE5D80709F485C0D8
:1034200078F4C330ECE5DE0709F478C008F07AC020
:10343000C230DC4509F0F5C08091B2028160EFC076
:10344000C7309CE5D90709F478C008F07AC08091AC
:10345000B2028061E4C0CD30FCE5DF0709F487C02B
:1034600058F4CB309CE5D90709F479C008F07BC04B
:103470008091B20288606FC0CF30FCE5DF0709F4AD
:1034800080C008F082C08091B202877FC8C0CE3F62
:103490009CE5D90709F471C000F5C531FCE5DF07EB
:1034A00009F485C068F4C3319CE5D90709F475C0F7
:1034B00008F095C00E94D00B8091B2028F77AFC008
:1034C000CC3FFCE5DF07A9F108F054C0CB3FDC4559
:1034D00009F0A7C08091B30240C0C230EDE5DE071D
:1034E00009F489C058F4C1158DE5D80709F45AC00C
:1034F00008F069C08091B30282602FC0C236EDE54A
:10350000DE0709F47CC0C63AFDE5DF0709F481C097
:10351000C330DD4509F085C080E06EC08091B20205
:1035200082607DC08091B20216C08091B202886034
:1035300076C08091B30282604FC08091B2028062F7
:103540006EC08091B20280646AC00E94D00B8091EC
:10355000B202806864C0846062C081603DC08091B6
:10356000B2028E7F5CC08091B2028D7F58C0809184
:10357000B20216C08091B30218C08091B3028D7F51
:103580002BC08091B2028F7E4AC08091B2028F7DA3
:1035900046C08091B2028F7B42C08091B202877F89
:1035A0008B7F3DC08091B3028D7F8E7F15C080914F
:1035B000B20282FB222720F991E0922790FB82F948
:1035C00090FB83F92CC08091B302982F9095917055
:1035D0008E7F892B90FB81F98093B30222C00E94D9
:1035E000D00B8091B20287FB222720F991E092272D
:1035F00090FB87F914C081E00E94C41212C0809130
:10360000B20284FB222720F991E0922790FB84F9F3
:1036100006C08091B202982F909590FB80F980931C
:10362000B2028091B2029091B3020E943E120E94B7
:10363000D00B80E001C081E0DF91CF910895089523
:1036400008958BEE0E94EA1C8A3FA1F40E94D51CCB
:103650009091B002892B809366020E94D51C8093C2
:1036600067020E94D51C90916702209166029923FF
:1036700049F014C08091500283FFB1C086ED91E003
:103680000C94A80581110AC030916902311106C05D
:10369000309164023227377009F497C02093640296
:1036A000322F307424FF07C031110AC0903841F026
:1036B00097FD09C005C0311105C097FF04C002C0C5
:1036C00091E801C09FE79093670225FF07C027FD9F
:1036D0000AC0803841F087FD09C005C027FD05C03C
:1036E00087FF04C002C081E801C08FE7922F977066
:1036F000909366028195809368028091630222FF15
:1037000027C0811109C00E94D9239093620280933F
:10371000610281E080936302909167028091680268
:10372000911102C08823C1F122E02093630287FD3A
:103730008F5F8595819580936902892F97FD8F5FB3
:10374000859580936A02109267021092680224C0E5
:10375000813001F580916102909162020E94F12313
:103760008C329140B8F48091660284608093660246
:1037700085E692E00E94BC228FEF91EE24E081501A
:1037800090402040E1F700C00000809166028B7FEE
:103790008093660210926302809166028B7F809311
:1037A000660280916702811108C0809168028111D0
:1037B00004C080916902882321F085E692E00E948E
:1037C000201B85E692E00E94BC22109267021092B4
:1037D00068021092690210926A02109266020895BD
:1037E000CF9384EF0E94EA1CC82F8091500283FF80
:1037F0001BC086EB91E00E94A80580918D021F926C
:103800008F931F92CF931F9284EF8F9380E991E063
:103810009F938F930E9441068DB79EB708960FB66F
:10382000F8949EBF0FBE8DBFCF910895CF930E9495
:10383000C21C2FEF83ED90E3215080409040E1F7D0
:1038400000C000008FEF0E94EA1CC82F8091500238
:1038500083FF1BC087E892E00E94A80580918D023B
:103860001F928F931F92CF931F928FEF8F9381E6BA
:1038700092E09F938F930E9441068DB79EB7089662
:103880000FB6F8949EBF0FBE8DBF0E94D51CC82FE7
:103890008091500283FF16C088E492E00E94A80540
:1038A00080918D021F928F931F92CF938FE292E0AF
:1038B0009F938F930E9441060F900F900F900F904F
:1038C0000F900F900E94D51CC82F8091500283FF4B
:1038D00016C084E192E00E94A80580918D021F929B
:1038E0008F931F92CF938BEF91E09F938F930E94C2
:1038F00041060F900F900F900F900F900F900E9425
:10390000F01BCF910C941F1B9FB7F89420916B0272
:1039100080916C02821761F030E0F901E359FD4FAC
:1039200080812F5F3F4F2F71332720936B0201C09F
:1039300080E09FBF0895CF93DF93EC010E94191E92
:10394000882341F0209731F085E08A95F1F7000057
:103950002197F4CFCE01DF91CF910895CF93DF93DC
:10396000C2E3D0E00E94191E811108C0209731F0F7
:1039700085E08A95F1F700002197F4CFCE01DF9121
:10398000CF9108950E94161E0E94271E5D985A9896
:1039900086E78093CA001092C8001092CD00109262
:1039A000CC0080E98093C90008958AE1815011F428
:1039B0000C94841C3FB7F89420916C0290916B0298
:1039C0003FBF2913F5CFEFE9FFE03197F1F700C0D2
:1039D0000000ECCFEF92FF920F931F93CF93DF93F2
:1039E000E82E10928D021092CA008091C900877E45
:1039F0008093C9000E94131E0E94271E8FE891E049
:103A00000197F1F700C000000E94241E0E94161EBC
:103A100080E197E20E949B1C892B11F48AE077C019
:103A2000C0E0D0E011E0F12C01E090E59A95F1F7CB
:103A3000C7010C2E02C0959587950A94E2F780FF86
:103A400004C010270E94271E02C00E94241E0E944C
:103A5000AE1C892B11F482E05AC082E390E00E94F0
:103A60009B1C892B11F483E052C02196C830D105EC
:103A7000E1F680E58A95F1F7112319F00E94271EDF
:103A800002C00E94241E0E94AE1C892B11F484E007
:103A90003EC082E390E00E949B1C892B11F485E0DC
:103AA00036C090E59A95F1F70E94271EC2E3D0E058
:103AB0000E942A1E882341F0209741F025E02A9594
:103AC000F1F700002197F4CFCD2B11F486E01FC051
:103AD00082E390E00E949B1C892B11F487E017C0C1
:103AE0000E94AE1C892B19F0C2E3D0E009C088E027
:103AF0000EC0209759F085E08A95F1F700002197D4
:103B00000E942A1E8823A9F3CD2BE9F489E0809333
:103B10008D020E94161E0E94271E5D985A9886E705
:103B20008093CA001092C8001092CD001092CC0071
:103B300080E98093C90080E0DF91CF911F910F91C0
:103B4000FF90EF9008950E94161E0E94271E5D9818
:103B50005A9886E78093CA001092C8001092CD0050
:103B60001092CC0080E98093C900DF91CF911F9122
:103B70000F91FF90EF900C94D51C1F920F920FB6EF
:103B80000F9211242F933F934F935F936F937F93E3
:103B90008F939F93AF93BF93CF93EF93FF938091B6
:103BA000C8008C714091CE0081111BC0CFB7F89432
:103BB00080916C0290E09C012F5F3F4F2F71332763
:103BC00050916B02521739F0FC01E359FD4F4083CD
:103BD00020936C0204C085EA92E00E94A805CFBF42
:103BE00010C01F924F931F928F9381EB92E09F938F
:103BF0008F930E9441060F900F900F900F900F909F
:103C00000F90FF91EF91CF91BF91AF919F918F91C5
:103C10007F916F915F914F913F912F910F900FBEC8
:103C20000F901F9018955D98559A089555985D9A34
:103C3000089555985D9A85E08A95F1F7000089B15D
:103C400085FB882780F908955A98529A08955298CA
:103C50005A9A089552985A9A85E08A95F1F7000089
:103C600089B182FB882780F90895809104011F9211
:103C70008F93809105011F928F93809108011F926D
:103C80008F93809109011F928F9380910A011F9257
:103C90008F9380910B011F928F9383ED92E09F93FE
:103CA0008F930E9441068DB79EB70E960FB6F8947B
:103CB0009EBF0FBE8DBF0895883220F58E3108F06B
:103CC00068C08B3091F1C0F4873009F0BEC081E04C
:103CD00080930B0184E180930A018AE080930901BB
:103CE0008EE18093080188E08093050188E280934B
:103CF000040185E394E0C6C0833109F443C08431F4
:103D000069F1A3C08F3409F49EC028F4893231F1DF
:103D1000883359F09AC0813531F008F4D4C0823527
:103D200009F4A7C092C08FEFA5C087E594E00E9478
:103D3000A8050E94351E1F9281E08F931F9288E094
:103D40008F9380E593E09F938F930E9441060F909D
:103D50000F900F900F900F900F9096C084E594E015
:103D60000E94A80580919202882309F4AAC01092AB
:103D70009202109291021092900210928F02109271
:103D80008E02B1C086E494E00E94A8050E94351E10
:103D90007BC08D5180939202833031F170F4813079
:103DA000D1F0823009F03FC08AE091E09093910217
:103DB000809390028BE891E01FC0853059F108F1A3
:103DC000863089F584E091E090939102809390028F
:103DD00086EC91E011C08BE091E09093910280938A
:103DE000900282E891E008C089E091E0909391020E
:103DF0008093900287E991E090938F0280938E02E6
:103E000018C088E091E0909391028093900284EA38
:103E100091E0F2CF85E091E090939102809390023F
:103E200083EB91E0E9CF1092920283E494E00E9448
:103E3000A80580919202882309F455C01F928F93A0
:103E40008FE394E00DC08AE015C082E394E01AC0CD
:103E500097FF47C0108280811F928F938CE294E07D
:103E60009F938F930E9441060F900F900F900F9099
:103E70000BC081E0E0919002F0919102309729F51A
:103E800089E294E00E94A80520919202222359F130
:103E900080918E0290918F02009711F48EE791E04D
:103EA0009F938F931F922F9380E294E09F938F9321
:103EB0000E9441060F900F900F900F900F900F905F
:103EC00016C080E0089586EFD5CF2081082E000C23
:103ED000990B820F911D8F3F910509F00CF4B8CF1B
:103EE0008FEF8083B8CF8CE194E00E94A80581E039
:103EF0000895CF93C82F1F928F938DE694E09F93E0
:103F00008F930E94410681E090E0A0E0B0E0BC0108
:103F1000CD0104C0660F771F881F991FCA95D2F77D
:103F20000E94280C0F900F900F900F90CF910C943F
:103F3000D00BEF92FF920F931F93CF93DF938B31B0
:103F400009F4EDC008F08EC08B3009F4B1C008F060
:103F500078C0863009F4AFC020F4853009F4BDC0C4
:103F60004EC1873009F4C0C0883009F048C10E94B2
:103F700029121F928F9382E998E09F938F930E945A
:103F800041060E94251283FB992790F91F929F9367
:103F900082FB992790F91F929F9381FB992790F9B3
:103FA0001F929F93982F91701F929F931F928F93B0
:103FB00089E498E09F938F930E9441060E942D12FE
:103FC00087FB222720F91F922F9386FB222720F9B7
:103FD0001F922F9385FB222720F91F922F9384FB9A
:103FE000222720F91F922F9383FB222720F91F926B
:103FF0002F9382FB222720F91F922F9391FB2227D8
:1040000020F91F922F93292F21701F922F9381FB4C
:10401000222720F91F922F93282F21701F922F9370
:104020009F938F9384E697E09F938F930E9441061E
:104030008DB79EB788960FB6F8949EBF0FBE8DBF02
:1040400035C0803109F495C020F48E3009F47BC06E
:10405000D6C0863109F4A8C0893109F0D0C08DEDF1
:1040600094E084C08A32E1F060F4873209F4C3C07E
:1040700028F48E3108F4C3C08D51BEC0893269F175
:10408000BEC0833448F48A3308F0B3C0853309F4E2
:10409000B2C0883369F0B3C0833409F4ACC0AFC098
:1040A0008DE399E00E94A8050E94C212C1E0ACC055
:1040B00081EC95E05BC080915002817F8E7F809380
:1040C00050028AE995E00E94A80589E399E00E94E0
:1040D000A80581E080939302E9CF8DE199E00E94E9
:1040E000A8050E94A106E2CF80915002C82FC0957A
:1040F000C170C0FB80F980935002CC2329F081E18C
:1041000099E00E94A80580C084E099E00E94A8057B
:1041100080915002897F877F80935002C7CF909112
:10412000500291FBCC27C0F981E0C827892FC0FB42
:1041300081F980935002CC2319F087EF98E029C0D1
:1041400089EE98E013C09091500292FBCC27C0F901
:1041500081E0C827892FC0FB82F980935002CC23CD
:1041600019F08AED98E015C08AEC98E00E94A80545
:104170009DCF9091500293FBCC27C0F981E0C827D6
:10418000892FC0FB83F980935002CC2351F08EEB32
:1041900098E00E94A80580915002816080935002AF
:1041A00033C081EB98E0E2CF0E94E523162F072F62
:1041B000F82EE92ED091AF02C09118010E9467221B
:1041C000EF92FF920F931F931F92DF931F92CF9353
:1041D0001F928F9382E794E09F938F930E944106F2
:1041E0008DB79EB70C960FB6F8949EBF0FBE8DBFCD
:1041F0005DCF895301C080E00E94791F57CF8FEABD
:1042000098E00E94A805C0E08C2FDF91CF911F910C
:104210000F91FF90EF90089580E008950C940C2189
:10422000CF93C82F80919302813071F040F082309B
:1042300009F045C08C2F0E945C1E81E046C00E94A0
:1042400023118232F1F504C00E942311823261F4FD
:104250008C2F0E940E21811104C08C2F0E94991F67
:104260002CC081E090E029C08C2F0E940C2181118C
:1042700023C0C431C9F058F4CB3069F0C031B9F46F
:1042800082E08093930288E30E945C1E15C0C932CD
:1042900059F0C83361F48AE995E00E94A80589E6DF
:1042A00094E00E94A80508C0109293020CC087E613
:1042B00094E00E94A80507C081E0817006C01092BA
:1042C000930280E002C080E0F8CFCF910895CF93B1
:1042D000DF9386319C4541F5EB010E942311982F15
:1042E0008A812091020130910301882379F09A7A22
:1042F00081E009F480E080939402911102C069E2A8
:1043000001C065E3C9010E9438230AC0809194026C
:10431000811102C069E201C065E3C9010E943A232C
:104320000E94651180E001C081E0DF91CF91089586
:104330000F931F93CF93DF93C42FD22FFC01828161
:104340008823C9F0409397020E94D9239093960244
:104350008093950280E28C0F883008F057C0C770B8
:1043600081E001C0880FCA95EAF7DF91CF911F91D4
:104370000F910C941F0980919702481330C08091CF
:104380009502909196020E94F123883C910538F5A0
:1043900010E21D0FCD17B9F080E28C0F883040F489
:1043A000C77081E001C0880FCA95EAF70E9426090C
:1043B000183028F581E09D2F977001C0880F9A95DD
:1043C000EAF70E941F09802F0E9416091830F0F4A6
:1043D000D77081E001C0880FDA95EAF70AC080E261
:1043E0008C0F883098F4C77081E001C0880FCA959F
:1043F000EAF7DF91CF911F910F910C942609802F3E
:10440000DF91CF911F910F910C941609DF91CF91FD
:104410001F910F9108950F939C01CB01243F4CE510
:10442000340731F188F4293DFCE53F07D9F02A3DF6
:104430004CE5340779F1283D3C45A9F506E221EE2B
:1044400041EE68ED7CE52BC0263FFCE53F07E1F03F
:10445000A8F0273F3C4539F507E225EE46EE67EF29
:104460007CE51DC007E225EE45EE69ED7CE517C051
:1044700006E221EE40EE64EF7CE511C007E225EE96
:1044800044EE65EF7CE50BC006E221EE42EE66EFFE
:104490007CE505C008E221E045EE6AED7CE50E947E
:1044A000982180E008C0FC018281882319F01092D5
:1044B000970201C081E00F9108959093EB018093E2
:1044C000EA01089590939D0280939C020895E091E3
:1044D0009C02F0919D02309721F00190F081E02D37
:1044E000099480E00895EF92FF920F931F93CF936A
:1044F000DF93E0919C02F0919D023097B1F18C0125
:104500000280F381E02D09958091500282FF2DC039
:1045100080FF04C086E599E00E94A805E80118E044
:1045200080E5E82E89E0F82E8091500280FF0BC0D4
:1045300088811F928F93FF92EF920E9441060F9005
:104540000F900F900F90115021961111EDCF809187
:10455000500280FF0AC08EE499E0DF91CF911F9155
:104560000F91FF90EF900C94A805DF91CF911F91D0
:104570000F91FF90EF900895E0919C02F0919D02C1
:10458000309739F022E0DC012C930480F581E02D96
:104590000994089520919A0230919B0228173907B7
:1045A00071F090939B0280939A02E0919C02F091AB
:1045B0009D02309721F00680F781E02D099408953F
:1045C00020919802309199022817390771F0909341
:1045D000990280939802E0919C02F0919D0230979D
:1045E00021F00084F185E02D09940895FC013296B4
:1045F00097E080E0915029F021912223D9F38F5F39
:10460000F9CF0895662349F0FC013296089621916E
:10461000621729F0E817F907D1F780E0089581E0E3
:1046200008959C01FC0132969FEF80E0419146176E
:1046300089F09F3F19F4411101C0982F8F5F863098
:10464000A9F79F3F39F0F901E90FF11D97FDFA95A0
:104650006283089508959C012A5F3F4FFC014281C7
:10466000461301C01282019682179307B9F7089585
:104670000C9411230C942B23029626E0FC0111923A
:104680002A95E9F7089508950C94432383E08093D5
:104690009E020C944423811102C081E001C082E09B
:1046A00080939E020C9444230C944B2381E08093CE
:1046B0009E020C9444230C94562308950C945D237D
:1046C0000C945E230C945D230C945D230C945D2369
:1046D0000E9464230E9456160E94622380E00E947A
:1046E000AB1591E0811101C090E0892F08950895E4
:1046F0001F920F920FB60F9211248F939F93AF9337
:10470000BF9380919F02811113C08091B602909156
:10471000B702A091B802B091B9024196A11DB11D96
:104720008093B6029093B702A093B802B093B902F7
:10473000BF91AF919F918F910F900FBE0F901F90DF
:1047400018958091BE02843031F10E9421071092A9
:104750009F0220E488E190E00FB6F894A89580933A
:1047600060000FBE2093600083B7817F846083BFA9
:1047700083B7816083BF7894889583B78E7F83BF2A
:104780000FB6F894A89580916000886180936000CE
:10479000109260000FBE08950E94D00B0C94250764
:1047A00082E084BD93E095BD9AEF97BD80936E0043
:1047B00008952FB7F8948091B6029091B702A09116
:1047C000B802B091B9022FBF08952FB7F894609145
:1047D000B6027091B7028091B8029091B9022FBFD2
:1047E00008959C014FB7F8948091B6029091B7025A
:1047F000A091B802B091B9024FBF821B930B0895EC
:1048000078941F920F920FB60F9211248F939F935B
:10481000AF93BF938091B6029091B702A091B80276
:10482000B091B9020196A11DB11D8093B60290937B
:10483000B702A093B802B093B902BF91AF919F9114
:104840008F910F900FBE0F901F901895F89481E0F4
:104850008093E00080E28093D800E9ECF0E01082E1
:104860008FE19EE40197F1F700C000001DBA10929D
:1048700068001CBC10BE1FBA10927A0010926E0025
:1048800010926F0010927100109272001082ECEB87
:10489000F0E0108214B817B81AB81DB810BA108218
:1048A00015B818B81BB81EB811BA0C94003F08957B
:1048B0008091AE020895089522E02093E9002FEF41
:1048C0003091E800215035FD06C035ED3A95F1F7FD
:1048D00000002111F5CF2091E80025FF0BC040E03A
:1048E00050E066E070E00E9444278091E8008E77F7
:1048F0008093E8000895CF93DF9321E02093E900AF
:104900002FEF3091E800215035FD06C035ED3A9586
:10491000F1F700002111F5CF2091E80025FF14C028
:10492000EC0140E050E068E070E00E944427809194
:10493000E8008E778093E80088E0FE01A6EAB2E006
:1049400001900D928A95E1F7DF91CF9108958093C0
:10495000A2027093A4026093A3028091BE028430ED
:1049600001F582E08093E9008FEF9091E80081509B
:1049700095FD06C095ED9A95F1F700008111F5CFF0
:104980008091E80085FF0DC040E050E063E070E0FA
:1049900082EA92E00E9444278091E8008E7780931B
:1049A000E8000895BC0184E00C94A724BC0183E0D6
:1049B0000C94A7248CE799E00E94A8058091BD0281
:1049C000811109C00E94D5280E9432298091E200FD
:1049D00084608093E200089588E799E00E94A8052A
:1049E0001092BD02089584E799E00E94A8050C94F6
:1049F0005B2380E799E00E94A8056091BA0281E0FC
:104A0000611101C080E00C9446238CE699E00E947D
:104A1000A8059091BE0281E0943009F080E0609199
:104A2000BA020C944B232091A1022F5F822F62E3E4
:104A30000E94E12B992319F02093A102089510926E
:104A4000A1028091A502882371F18091BE02843079
:104A500041F58091E9008F702091EC00922F9170C8
:104A600020FD90E8892B93E09093E9009091EB0072
:104A700090FF14C09091EE0097FF10C09091E80055
:104A800095FF03C01092F100F9CF9091E80090FFDC
:104A900005C09091E8009E779093E8008F70809316
:104AA000E9001092A502089542E061EC81E00E94C5
:104AB0004E2842E261EC82E00E944E2842E261EC24
:104AC00083E00E944E289091BE0281E0943009F06C
:104AD00080E06091BA020C9454238091C00283302C
:104AE00009F461C030F4813071F0823009F49AC069
:104AF00008958A3009F486C08B3009F46CC089307F
:104B000009F0A8C020C08091BF02813A09F0A2C07C
:104B10008091E800877F8093E8008091C3029091A4
:104B2000C402892B21F468E086EA92E003C060E0C9
:104B300080E090E070E00E948F278091E8008B7702
:104B40008093E80008958091BF02813209F082C00D
:104B50008091C3029091C402029708F07BC08091BB
:104B6000E800877F8093E8008091E80082FD05C01F
:104B70008091BE028111F8CF6DC02091F300809129
:104B8000F20090E0922B029731F48091F100813095
:104B900011F0863021F48091F1008093AE02809173
:104BA000E8008B7753C08091BF02813A09F052C070
:104BB0008091C3029091C402892B09F04BC080916F
:104BC000E800877F8093E8008091E80080FFFCCFB9
:104BD0008091180136C08091BF028132D9F5809151
:104BE000C3029091C402892BA9F58091E800877FC8
:104BF0008093E8000E9483288091C102809318016D
:104C00000C94D00B8091BF02813221F58091E80095
:104C1000877F8093E8000E9483288091C20280935E
:104C2000AF0208958091BF02813AA1F48091E8001B
:104C3000877F8093E8008091E80080FFFCCF80911F
:104C4000AF028093F1008091E8008E778093E800B6
:104C50000C94832808959FB7F8941092A5029FBFE3
:104C60009091BE02943009F057C09091E9009F7076
:104C70003091EC00232F217030FD20E8922B23E0AF
:104C80002093E9002091EB0020FF43C02091EE002B
:104C900027FF3FC02091A002222321F02091E800AD
:104CA00025FF37C01092A00226E03091E80035FDC4
:104CB00015C03091BE02343061F53091EB0035FD06
:104CC00028C0215021F481E08093A00222C0EFE9A6
:104CD000FFE03197F1F700C00000E7CF8093F100CB
:104CE0008091E80085FD0AC08091E80080FFFCCF3C
:104CF0008091E8008E778093E80006C08FB7F89423
:104D000021E02093A5028FBF9F709093E90080E07F
:104D100008959F709093E9008FEF089584B7877F7F
:104D200084BF0FB6F894A895809160008861809345
:104D30006000109260000FBE90E080E80FB6F8941B
:104D400080936100909361000FBE0C9456230E94E3
:104D5000D5280E943229E2EEF0E0808184608083D1
:104D600078940C94C62B8CE091E00C946222809194
:104D7000BE028530C9F488E699E00E94A8058091BA
:104D8000BE02853079F40E94A1238091BC02882361
:104D9000B1F30E946823882391F30E942E270E947A
:104DA000D00BEDCF0C94CC23089508950C94D82605
:104DB000292F332723303105C9F060F42130310524
:104DC00081F02230310509F041C08BE590E020EB05
:104DD00039E040C021323105E1F02232310531F1B4
:104DE00035C082E190E02BE03AE034C09927813071
:104DF000910549F028F0029749F5E0E8F9E005C08F
:104E0000ECEAF9E002C0E2EAF9E0849190E09F0167
:104E100021C063307105D0F4660F771FFB01EC51A0
:104E2000FE4F2081318189E090E014C0633071052C
:104E300068F4FB01EE0FFF1FE252FE4F208131812B
:104E4000FB01E552FE4F808190E004C080E090E0DD
:104E500020E030E0FA0131832083089580E189BDAC
:104E600082E189BD09B400FEFDCF8091D8008F7D1D
:104E70008093D8008091E00082608093E000809170
:104E8000E00081FDFCCF0895CF92DF92EF92FF9278
:104E90000F931F93CF93DF93EC018B017A010E9454
:104EA000A228811133C0E114F10439F0F7018081A7
:104EB0009181081B190BC80FD91FC12CD12C0115CA
:104EC000110519F18091E80085FD16C08091E80078
:104ED0008E778093E800E114F10449F0F7018081B6
:104EE0009181C80ED91ED182C08285E00FC00E9478
:104EF000A228882321F30AC089918093F1000150F0
:104F00001109FFEFCF1ADF0ADACF80E0DF91CF91EE
:104F10001F910F91FF90EF90DF90CF900895209117
:104F2000C5023091C6022617370748F06115710592
:104F300039F42091E8002E772093E80001C0B901F0
:104F4000FC0120E06115710579F18091BE02882392
:104F5000F1F18530F1F18091E80083FD3CC0809152
:104F6000E80082FD2EC08091E80080FFEBCF209109
:104F7000F3008091F20090E0922B6115710551F0E1
:104F80008830910538F421912093F1006150710926
:104F90000196F3CF21E0089709F020E08091E80026
:104FA0008E778093E800CECF2111CFCF0AC08091B9
:104FB000BE02882361F0853061F08091E80083FDB6
:104FC0000AC08091E80082FFF2CF80E0089582E07D
:104FD000089583E0089581E008952091C5023091FD
:104FE000C6022617370748F06115710539F420917C
:104FF000E8002E772093E80001C0B901FC0120E011
:105000006115710591F18091BE02882309F440C0B9
:10501000853009F43FC08091E80083FD3DC0809158
:10502000E80082FD2FC08091E80080FFE9CF209149
:10503000F3008091F20090E0922B6115710559F018
:105040008830910540F424912093F100319661500D
:1050500071090196F2CF21E0089709F020E08091D4
:10506000E8008E778093E800CBCF2111CCCF0AC027
:105070008091BE02882361F0853061F08091E80064
:1050800083FD0AC08091E80082FFF2CF80E008959E
:1050900082E0089583E0089581E00895982F973085
:1050A00068F59093E900981739F07091EC00209121
:1050B000ED005091F00003C0242F762F50E021FD29
:1050C00002C09F5FECCF3091EB003E7F3093EB004E
:1050D0003091ED003D7F3093ED003091EB00316079
:1050E0003093EB007093EC002093ED005093F000B0
:1050F0002091EE0027FDE5CF80E008958F7080932A
:10510000E90081E008958091BF0287FF11C080917E
:10511000E80082FD05C08091BE028111F8CF11C068
:105120008091E8008B770BC08091BE02882349F004
:105130008091E80080FFF8CF8091E8008E7780931F
:10514000E80008952091E4003091E50095E6409153
:10515000EC00842F817040FF23C08091E80080FD27
:105160001DC08091BE02882399F0853099F080910E
:10517000EB0085FD11C04091E4005091E50024173B
:10518000350729F3915011F09A01E1CF84E0089599
:1051900082E0089583E0089581E0089580E0089515
:1051A0004091E80042FFDDCF08950E9443290E940C
:1051B0004B29E0EEF0E0808181608083E8EDF0E053
:1051C00080818F77808319BCA7EDB0E08C918E7FB2
:1051D0008C9380818F7E80831092BD0208950F93FF
:1051E0001F93CF93DF930E9443290E944B29C8ED60
:1051F000D0E088818F7788838881806888838881E0
:105200008F7D888319BC1092BE021092BA02109250
:10521000BC021092BB0200EE10E0F80180818B7F8F
:10522000808388818160888342E060E080E00E9422
:105230004E28E1EEF0E080818E7F8083E2EEF0E0A8
:10524000808181608083808188608083F801808193
:105250008E7F8083888180618883DF91CF911F91C9
:105260000F910895E8EDF0E080818F7E8083E7ED77
:10527000F0E080818160808384E082BF81E0809360
:10528000BD020C94EF28E8EDF0E080818E7F8083F2
:105290001092E20008951092DA001092E100089551
:1052A0001F920F920FB60F9211242F933F934F939B
:1052B0005F936F937F938F939F93AF93BF93EF937E
:1052C000FF938091E10082FF0BC08091E20082FF9A
:1052D00007C08091E1008B7F8093E1000E9413253D
:1052E0008091DA0080FF1FC08091D80080FF1BC032
:1052F0008091DA008E7F8093DA008091D90080FF60
:105300000DC080E189BD82E189BD09B400FEFDCFF9
:1053100081E08093BE020E94DA2405C019BC10927D
:10532000BE020E94EC248091E10080FF19C08091B0
:10533000E20080FF15C08091E2008E7F8093E20042
:105340008091E20080618093E2008091D8008062C9
:105350008093D80019BC85E08093BE020E94F92496
:105360008091E10084FF30C08091E20084FF2CC076
:1053700080E189BD82E189BD09B400FEFDCF809145
:10538000D8008F7D8093D8008091E1008F7E80933C
:10539000E1008091E2008F7E8093E2008091E20044
:1053A00081608093E2008091BA02882311F084E04A
:1053B00007C08091E30087FD02C081E001C083E067
:1053C0008093BE020E9405258091E10083FF29C0E1
:1053D0008091E20083FF25C08091E100877F809368
:1053E000E10082E08093BE021092BA028091E10057
:1053F0008E7F8093E1008091E2008E7F8093E200B7
:105400008091E20080618093E20042E060E080E011
:105410000E944E288091F00088608093F0000E94E6
:10542000F324FF91EF91BF91AF919F918F917F9165
:105430006F915F914F913F912F910F900FBE0F9001
:105440001F9018951F920F920FB60F9211242F9351
:105450003F934F935F936F937F938F939F93AF93FC
:10546000BF93CF93DF93EF93FF93C091E900CF7089
:105470008091EC00D82FD17080FDD0E81092E90027
:105480008091F000877F8093F00078940E94662AD4
:105490001092E9008091F00088608093F000CD2B9D
:1054A000CF70C093E900FF91EF91DF91CF91BF9151
:1054B000AF919F918F917F916F915F914F913F91AC
:1054C0002F910F900FBE0F901F9018951F93CF93A1
:1054D000DF93CDB7DEB7AA970FB6F894DEBF0FBE45
:1054E000CDBFEFEBF2E08091F100819322E0E73C49
:1054F000F207C9F70E946D258091E80083FF2EC155
:105500008091BF029091C002492F50E04A3051056E
:1055100008F024C1FA01EE59FF4F0C94012C803899
:1055200021F0823809F01AC108C08091BB02909125
:10553000BC02992389F082600FC08091C3028F70F2
:10554000873008F00BC18093E9008091EB0085FB68
:10555000882780F91092E9009091E800977F909356
:10556000E8008093F1001092F100D1C0282F2D7F28
:1055700009F0F4C0882319F0823061F0EFC0809107
:10558000C102813009F0EAC0933009F080E08093D5
:10559000BC022EC08091C10281112AC08091C30239
:1055A0008F702FEF280F263008F0D8C08093E900C5
:1055B0002091EB0020FF1CC0933021F48091EB0080
:1055C000806214C09091EB0090619093EB0021E019
:1055D00030E0A90102C0440F551F8A95E2F74093BD
:1055E000EA001092EA008091EB0088608093EB0063
:1055F0001092E9008091E800877F8093E8000E9484
:105600008328ACC08111AAC01091C1021F7780917C
:10561000E3008078812B8093E3008091E800877F0E
:105620008093E8000E9483288091E80080FFFCCFEF
:105630008091E30080688093E300111102C082E052
:1056400001C083E08093BE0289C08058823008F098
:1056500085C08091C1029091C2028C3D53E09507B4
:1056600079F583E08A838AE289834FB7F894DE0173
:10567000139620E03EE051E2E32FF0E05093570014
:10568000E49120FF03C0E295EF703F5FEF708E2F33
:1056900090E0EA3010F0C79601C0C0968D939D93BC
:1056A0002F5F243149F74FBF8091E800877F8093B7
:1056B000E8006AE270E0CE0101960E948F2716C0D2
:1056C0006091C3027091C402AE014F5F5F4F0E94B0
:1056D000D626BC01892B09F441C09091E800977F40
:1056E0009093E80089819A810E94ED278091E800DB
:1056F0008B778093E80032C0803881F58091E80094
:10570000877F8093E8008091BA028093F1008091B6
:10571000E8008E7772CF811121C08091C1029091F3
:10572000C20299270297D4F48091E800877F809382
:10573000E8008091C1028093BA020E948328809180
:10574000BA02811106C08091E30087FD02C081E0AA
:1057500001C084E08093BE020E9454258091E8003D
:1057600083FF0AC08091E800877F8093E8008091E2
:10577000EB0080628093EB00AA960FB6F894DEBF30
:105780000FBECDBFDF91CF911F910895CF93809130
:10579000BE028823A1F0C091E900CF709091EC0087
:1057A000892F817090FD80E8C82B1092E9008091CC
:1057B000E80083FD0E94662ACF70C093E900CF9174
:1057C0000895991B79E004C0991F961708F0961B5D
:1057D000881F7A95C9F78095089597FB072E16F4D0
:1057E000009407D077FD09D00E94072C07FC05D054
:1057F0003EF4909581959F4F0895709561957F4FE8
:105800000895EE0FFF1F0590F491E02D0994AA1B57
:10581000BB1B51E107C0AA1FBB1FA617B70710F09B
:10582000A61BB70B881F991F5A95A9F780959095CD
:10583000BC01CD010895FB01DC0104C08D910190F4
:10584000801921F441505040C8F7881B990B0895E6
:10585000F999FECF92BD81BDF89A992780B5089538
:10586000A8E1B0E042E050E00C945C2C262FF999BE
:10587000FECF92BD81BDF89A019700B4021639F0AF
:105880001FBA20BD0FB6F894FA9AF99A0FBE089580
:105890000396272F0E94372C0E94362C252F0E941A
:1058A000372C242F0C94372C0196272F0E94372C4D
:1058B0000C94362CDC01CB01FC01F999FECF06C01B
:1058C000F2BDE1BDF89A319600B40D9241505040BE
:0858D000B8F70895F894FFCF2A
:1058D800C8003D02280850011E0A140158247B24E0
:1058E8005C24D624D2245B2401E200E900EA00B556
:1058F80000B600B700CD008301CC008A0192019464
:10590800012102230224022502260227022A02B3C9
:1059180000B4006F007000818283E200E900EA00B1
:10592800B500B600B700CD008301CC008A01920112
:1059380094012102230224022502260227022A02B8
:10594800B300B4006F007000818283F1F4F53F3F2B
:105958003F006D6B5F64656C6179006D6B5F696EAC
:1059680074657276616C006D6B5F6D61785F7370E2
:10597800656564006D6B5F74696D655F746F5F6DFD
:105988006178006D6B5F776865656C5F6D61785FE6
:105998007370656564006D6B5F776865656C5F74CF
:1059A800696D655F746F5F6D617800407B22BA0A2C
:0A59B8003F0A1D0AC209DB09F409C9
:00000001FF
